:1000000012C0189518951895189518951895189563
:100010001895189518951895189518951895189578
:100020001895189518958FE58DBFC0E4E0E34E2E26
:1000300084E08EBFD4E0F4E05F2EEEEFF3E0A0E6C4
:10004000B0E088278D933197E9F789E189B980E09D
:1000500080BD88E18AB966248EE181BD86E181BDDB
:10006000A098A198A298A398A498A5988A9A8B9AE8
:100070008C9A8D9A8E9A8F9A929893989498959834
:100080009698979880E08093990080E080939E00F6
:100090008BE180939700A7E9B0E08C91A2E9B0E0F2
:1000A0008D9388278C93A2E9B0E000D6E2E8F3E1D3
:1000B00037D886D3E0E0F0E0AFE9B0E041D9E1E045
:1000C000F0E0A0EAB0E03CD9E2E0F0E0A1EAB0E084
:1000D00037D900919F000F3F09F00BC00091A0009D
:1000E0000F3F09F006C00091A1000F3F09F001C0C9
:1000F0005FD5E2E0F0E0FED548D562D305D30091AC
:100100009F00003009F013C181B5886081BDA198BE
:10011000A09898E1A0E6B0E0983018F4392F99271C
:1001200002C038E09850999BFECF88949899089423
:1001300087959999FECF3A95B1F78D93992361F7F9
:1001400000E010E020E030E0A0E6B0E00D931D9369
:100150002D933C93A198A09898E1A0E6B0E0983048
:1001600018F4392F992702C038E09850999BFECF98
:1001700088949899089487959999FECF3A95B1F704
:100180008D93992361F7A8957DD2BED200919E00F0
:10019000013009F00CC0EAE7F3E182D8EAE9F0E0C7
:1001A000D5D7DCD5EDE0F0E0AAE9B0E09DD800912C
:1001B0009900003009F08DC0A7E9B0E08C9196D588
:1001C000E6E8F3E18AD5A7E9B0E08C918FD5ECE8B9
:1001D000F3E183D5E0E9F3E180D5A7E8B0E077D596
:1001E000A8E1B4E0A8E1B4E0EAE9F0E0552742E094
:1001F0000BD66BD5EAE9F3E170D5A7E9B0E08C91B5
:1002000075D5EEE9F3E169D5A7E9B0E08C916ED53B
:10021000E2EAF3E162D5A7E9B0E08C9167D5E8EABC
:10022000F3E15BD5E0E9F3E158D5A7E8B0E04FD5BD
:10023000A8E1B4E0A8E1B4E0EAE9F0E0552742E043
:10024000E3D543D5EAE9F3E148D5A7E9B0E08C91DD
:100250004DD5EEE9F3E141D5A7E9B0E08C9146D563
:10026000ECEAF3E13AD5E4EBF3E137D500919E00F7
:10027000013009F015C0A7E9B0E08C9137D5E6EB65
:10028000F3E12BD5EEEBF3E128D5A7E9B0E08C91B3
:100290002DD5ECEAF3E121D5E4EBF3E11ED518C04E
:1002A000A7E9B0E08C9122D5E6EBF3E116D5A7E9FA
:1002B000B0E08C911BD5EEE9F3E10FD5A7E9B0E0F2
:1002C0008C9114D5ECEAF3E108D5E4EBF3E105D524
:1002D0002EC0A7E9B0E08C9109D5E6E8F3E1FDD4A2
:1002E000E4ECF3E1FAD4A8E1B4E0E0E6F0E0EAD728
:1002F000ECD4A7E9B0E08C91F9D4A7E9B0E08C91F7
:10030000F5D4E2EAF3E1E9D4E4ECF3E1E6D4A8E1E0
:10031000B4E0E0E6F0E0D6D7D8D4A7E9B0E08C911D
:10032000E5D4ECEAF3E1D9D4E4EBF3E1D6D40091DF
:10033000A000003009F0D0C081B5886081BDA398CD
:10034000A29898E1A0E6B0E0983018F4392F9927E8
:1003500002C038E098509B9BFECF88949A990894ED
:1003600087959B99FECF3A95B1F78D93992361F7C5
:1003700000E010E020E030E0A0E6B0E00D931D9337
:100380002D933C93A398A29898E1A0E6B0E0983012
:1003900018F4392F992702C038E098509B9BFECF64
:1003A00088949A99089487959B99FECF3A95B1F7CE
:1003B0008D93992361F7A89565D1A6D100919900F5
:1003C000003009F05BC0A7E9B0E08C918FD4EEEC6F
:1003D000F3E183D4A7E9B0E08C9188D4ECE8F3E1B1
:1003E0007CD4E4EDF3E179D4A7E8B0E070D4A8E1DF
:1003F000B4E0A8E1B4E0EAE9F0E0552742E004D532
:1004000064D4EAE9F3E169D4A7E9B0E08C916ED451
:10041000EEE9F3E162D4A7E9B0E08C9167D4EEEDA8
:10042000F3E15BD4A7E9B0E08C9160D4E8EAF3E1B2
:1004300054D4E4EDF3E151D4A7E8B0E048D4A8E106
:10044000B4E0A8E1B4E0EAE9F0E0552742E0DCD40A
:100450003CD4EAE9F3E141D4A7E9B0E08C9146D479
:10046000EEE9F3E13AD4A7E9B0E08C913FD4ECEAAD
:10047000F3E133D4E4EBF3E130D42EC0A7E9B0E0EC
:100480008C9134D4EEECF3E128D4E4EEF3E125D4FE
:10049000A8E1B4E0E0E6F0E015D717D4A7E9B0E0B2
:1004A0008C9124D4A7E9B0E08C9120D4EEEDF3E157
:1004B00014D4E4EEF3E111D4A8E1B4E0E0E6F0E016
:1004C00001D703D4A7E9B0E08C9110D4ECEAF3E1B2
:1004D00004D4E4EBF3E101D40091A100003009F071
:1004E000D0C081B5886081BDA598A49898E1A0E6A8
:1004F000B0E0983018F4392F992702C038E09850AE
:100500009D9BFECF88949C99089487959D99FECFDA
:100510003A95B1F78D93992361F700E010E020E060
:1005200030E0A0E6B0E00D931D932D933C93A59889
:10053000A49898E1A0E6B0E0983018F4392F9927F4
:1005400002C038E098509D9BFECF88949C990894F7
:1005500087959D99FECF3A95B1F78D93992361F7D1
:10056000A89590D0D1D000919900003009F05BC0DF
:10057000A7E9B0E08C91BAD3EEEEF3E1AED3A7E9F0
:10058000B0E08C91B3D3ECE8F3E1A7D3E6EFF3E16D
:10059000A4D3A7E8B0E09BD3A8E1B4E0A8E1B4E01D
:1005A000EAE9F0E0552742E02FD48FD3EAE9F3E1FE
:1005B00094D3A7E9B0E08C9199D3EEE9F3E18DD320
:1005C000A7E9B0E08C9192D3E0E0F4E186D3A7E90B
:1005D000B0E08C918BD3E8EAF3E17FD3E6EFF3E16F
:1005E0007CD3A7E8B0E073D3A8E1B4E0A8E1B4E01D
:1005F000EAE9F0E0552742E007D467D3EAE9F3E1FE
:100600006CD3A7E9B0E08C9171D3EEE9F3E165D347
:10061000A7E9B0E08C916AD3ECEAF3E15ED3E4EBB6
:10062000F3E15BD32EC0A7E9B0E08C915FD3EEEE8F
:10063000F3E153D3E8E0F4E150D3A8E1B4E0E0E61D
:10064000F0E040D642D3A7E9B0E08C914FD3A7E9C0
:10065000B0E08C914BD3E0E0F4E13FD3E8E0F4E18B
:100660003CD3A8E1B4E0E0E6F0E02CD62ED3A7E935
:10067000B0E08C913BD3ECEAF3E12FD3E4EBF3E170
:100680002CD33DCD94E0A0E6B0E04FD5A4E6B0E099
:10069000E0E6F0E017D684E1E4E6F0E001E00A935A
:1006A000A5E8B0E027D6A5E8B0E0E2E1F4E152D653
:1006B00009F017C00FEF1FEF2FE030E0A0E6B0E029
:1006C0004D915D916D917C91F4D5A0E6B0E00D93D4
:1006D0001D932D933D93A7E8B0E0E4E1F4E120D52C
:1006E00005C0A7E8B0E0E6E1F4E11AD5EEE7F3E1F2
:1006F000D7D5E0E6F0E02AD53BD578D5EDE0F0E0BF
:10070000AAE9B0E0F1D50895D8D2A8E9B0E08C9379
:1007100000919800003010F009F001C03FC082E65F
:10072000482F00919800041709F003C081E08093DE
:10073000990083E6482F00919800041709F001C042
:10074000BED184E6482F00919800041709F006C036
:1007500080E08093990080E080939E0085E6482F9A
:1007600000919800041709F001C022D286E6482FB4
:1007700000919800041709F001C076D182E7482F54
:1007800000919800041709F003C081E080939E0057
:10079000009198000B3109F001C012D0A7E9B0E038
:1007A0008C91A4D2ECEAF3E198D2E4EBF3E195D298
:1007B000A7E9B0E08C919AD2EEE9F3E18ED20895E8
:1007C000A2E9B0E084D2A7E9B0E08C918FD2E8E151
:1007D000F4E183D2E0E2F4E180D285D2A7E9B0E08F
:1007E0008C9184D2EAE5F4E178D2E2E6F4E175D2C4
:1007F0007AD2A7E9B0E08C9179D2E6E8F3E16DD244
:10080000A7E9B0E08C9172D2ECE8F3E166D2E0E9BE
:10081000F3E163D2A7E9B0E08C9168D2E2EAF3E1B8
:100820005CD2A7E9B0E08C9161D2E8EAF3E155D25D
:10083000E0E9F3E152D2A7E9B0E08C9157D2EEECB7
:10084000F3E14BD2A7E9B0E08C9150D2ECE8F3E1B0
:1008500044D2E4EDF3E141D2A7E9B0E08C9146D275
:10086000EEEDF3E13AD2A7E9B0E08C913FD2E8EAAD
:10087000F3E133D2E4EDF3E130D2A7E9B0E08C91BB
:1008800035D2EEEEF3E129D2A7E9B0E08C912ED279
:10089000ECE8F3E122D2E6EFF3E11FD2A7E9B0E002
:1008A0008C9124D2E0E0F4E118D2A7E9B0E08C9179
:1008B0001DD2E8EAF3E111D2E6EFF3E10ED2A7E9A7
:1008C000B0E08C9113D2EAE7F4E107D2E2E8F4E178
:1008D00004D2A7E9B0E08C9109D2E4EAF4E1FDD1B9
:1008E000ECEAF4E1FAD1A7E9B0E08C91FFD1EEECAB
:1008F000F4E1F3D1E6EDF4E1F0D1A7E9B0E08C91B9
:10090000F5D1E8EFF4E1E9D1E0E0F5E1E6D1A7E9DE
:10091000B0E08C91EBD1E2E2F5E1DFD1EAE2F5E182
:10092000DCD1A7E9B0E08C91E1D1ECE4F5E1D5D1DF
:10093000E4E5F5E1D2D1A7E9B0E08C91D7D1E6E7C3
:10094000F5E1CBD1EEE7F5E1C8D1A7E9B0E08C91B4
:10095000CDD1E0EAF5E1C1D1E8EAF5E1BED1A7E900
:10096000B0E08C91C3D1EAECF5E1B7D1E2EDF5E16D
:10097000B4D1A7E9B0E08C91B9D1ECEAF3E1ADD103
:10098000E4EBF3E1AAD1A7E9B0E08C91AFD1EEE9B5
:10099000F3E1A3D100919F000F3F09F01EC0A7E92A
:1009A000B0E08C91A3D1E6E8F3E197D1E4EFF5E173
:1009B00094D1A7E9B0E08C9199D1E2EAF3E18DD12D
:1009C000E4EFF5E18AD1A7E9B0E08C918FD1ECEAB0
:1009D000F3E183D1E4EBF3E180D10091A0000F3F7C
:1009E00009F01EC0A7E9B0E08C9180D1EEECF3E1F4
:1009F00074D1E4E0F6E171D1A7E9B0E08C9176D151
:100A0000EEEDF3E16AD1E4E0F6E167D1A7E9B0E009
:100A10008C916CD1ECEAF3E160D1E4EBF3E15DD1D0
:100A20000091A1000F3F09F01EC0A7E9B0E08C9132
:100A30005DD1EEEEF3E151D1E4E1F6E14ED1A7E96B
:100A4000B0E08C9153D1E0E0F4E147D1E4E1F6E18C
:100A500044D1A7E9B0E08C9149D1ECEAF3E13DD172
:100A6000E4EBF3E13AD10895929A88E290E051D113
:100A7000929888EC90E04DD1939A88E290E049D129
:100A80009398A895959A88E290E043D1959888EC40
:100A900090E03FD1949A88E290E03BD19498A89559
:100AA000979A88E290E035D1979888EC90E031D120
:100AB000969A88E290E02DD19698A8950895A7E996
:100AC000B0E08C9113D1ECEAF3E107D1E4E2F6E176
:100AD00004D1A7E9B0E08C9109D1EEE9F3E1FDD0B2
:100AE000ECD0A8E9B0E08C93A89500919800003074
:100AF00010F009F001C02FC08AE7482F009198003C
:100B0000041709F006C0939A8CE291E002D1939801
:100B1000A89589E7482F00919800041709F006C0AE
:100B2000949A8CE291E0F5D09498A89588E7482FA4
:100B300000919800041709F006C0969A8CE291E0A3
:100B4000E8D09698A89581E6482F00919800041760
:100B500009F001C01AD000919800003010F009F09F
:100B600001C0BECFA7E9B0E08C91C0D0ECEAF3E1C0
:100B7000B4D0E4EBF3E1B1D0A7E9B0E08C91B6D00A
:100B8000EEE9F3E1AAD0A8950895939A8CE291E05A
:100B9000C0D09398A895949A8CE291E0BAD094989A
:100BA000A895969A8CE291E0B4D09698A89508956D
:100BB000A7E9B0E08C919AD0ECEAF3E18ED0E4EBB7
:100BC000F3E18BD0A7E9B0E08C9190D0EEE9F3E1AE
:100BD00084D0E8E4F6E181D070D0A8E9B0E08C934D
:100BE00000919800003010F009F001C055C088E76E
:100BF000482F00919800041709F00BC080E0809303
:100C00009F00E0E0F0E0A0E1BB2780E08C937BE771
:100C100086D389E7482F00919800041709F00BC08C
:100C200080E08093A000E1E0F0E0A0E1BB2780E05D
:100C30008C937BE774D38AE7482F009198000417C0
:100C400009F00BC080E08093A100E2E0F0E0A0E1B9
:100C5000BB2780E08C937BE762D38CE6482F009122
:100C60009800041709F018C0E0E0F0E0A0E1BB270D
:100C70008FEF8C937BE753D3E1E0F0E0A0E1BB275B
:100C80008FEF8C937BE74BD3E2E0F0E0A0E1BB2752
:100C90008FEF8C937BE743D3A895009198000D309C
:100CA00009F09ACF8DDD0895F894FFCF8F938D9141
:100CB0008823E9F711978F91089588275F9B0895FE
:100CC00000C05F9BFECF8CB10895A8E1B4E08D9188
:100CD000882311F00BD0FBCF0895DED2802D11F0C8
:100CE00005D0FBCF08958DE001D08AE05D9BFECF5B
:100CF0008CB9089588EE93E00CD03197D9F7089518
:100D00003197F1F70895689462F80895E89462F8CD
:100D10000895EF93FF93EE27E82BE92B31F0E0EAFB
:100D2000FFE03197F1F70197D1F7FF91EF91089527
:100D30008F939F93D216E306F4060FB680E890E8EF
:100D4000802795270FBE89070FB6892B87FD02C024
:100D500091E009260FBE9F918F91089543D0A9F08D
:100D6000503899F01627050F1BF40AF06CC272C2B6
:100D700003951BD0FF202AF0BB0CDD1CEE1CFF1CD2
:100D800002C003951BF003D0EBC164C25CC2B7FE86
:100D9000089590E8B91611F4D0FE08959FEFD91A7E
:100DA000E90AF90A09F403950895FF92EF928D2D4F
:100DB000FF24EE24DD24BB2493E0849F1001829F56
:100DC000B00CD11CE21CF31C839FD00CE11C22242C
:100DD000F21C9A9531F0BD2CDE2CEF2CFF248F9164
:100DE000ECCF0895652F90E8440F551F5927990FB0
:100DF00047956078102F90E8FF0C001F0927990F86
:100E0000F794107800380895A1D1F4DF17FF03C0DC
:100E10008DE28D931127003819F4E4ECF0E180C1E4
:100E20000F3741F4FF2019F4EAEBF0E1F8CFE6EBDD
:100E3000F0E1F5CF4A934A934A935A93BA93AA930F
:100E4000BB270F5FCAF4BB27802F0A9589D18D3E3F
:100E500070F4E4E1F1E1A3E023D26ADFBB1FB0FF4D
:100E600004C070971DD27ADF3C96AA95A9F7E0E1FD
:100E7000F1E116D273DF1DC0093028F1033148F1CA
:100E80000A3130F418E08BE192E9E8ECF0E128C097
:100E90000A9566D1E8E0F1E1BFEFA3E001D248DFB7
:100EA000BB1FB0FD04C03896FBD158DF3C97AA9514
:100EB000A9F7B095BB0F9EDF039513E08AEF99E089
:100EC000F816090740F413E08BE094E0ECEDF0E154
:100ED00007C016E001C0B39583E194E2E0EDF0E1D4
:100EE0006A81BF3F19F4BB2711276260BD836A8303
:100EF0001C83A881B98160E36D93A883B9836D9346
:100F0000081B0195AA24BB246A816A7F002339F05B
:100F1000F694E794D794B794A7940A95F7CF19E07D
:100F20000027BED1CC248FEF74E0AC14B206D306F8
:100F3000E406F50630F0AC18B20AD30AE40AF50A62
:100F400021F1881F7A9531F0569547953795279569
:100F5000C794EBCF809522D041F0969510F7FE2CE8
:100F6000ED2CDB2CBA2CAA24DCCF25D05D813C8172
:100F70002B8170D0277021F02BD06CD0E8F301C00A
:100F80003CD04CD078D0269608958894881F7A95C6
:100F9000E9F7809503D049F38827FCCF806360FD93
:100FA00006C0803311F0616002C0039561FD8D932E
:100FB00060FD1A95089599278E919C9385338E91A3
:100FC00008F083958A3308F080E38C93C0F7089586
:100FD000732F720F61FF701B0AD01296785019F0B0
:100FE00050F38E9380E38E937150EAF70895A881B1
:100FF000B981A70F8827B81F089579E061FD700FA8
:10100000F6DF48E0431B400F8AF381F399274A95A6
:1010100069F38E91803351F79C93F9CF732F61FF61
:10102000701B7395A881B981EA2FFB2F11978191CD
:10103000803361FF09F08D937A9511F48EE28D93E0
:1010400081918823C1F7772311F480E38D9388275A
:101050008C930895889462FD0895002359F4A88123
:10106000B9818C91803331F0552321F05395335061
:101070006460089408955523E9F085E48D931AF48B
:101080008DE28D935195652F660F560F5A3010F0F3
:1010900060E503D068E001D0DACF8FEF74E0561737
:1010A00008F0561B881F7A9511F06695F8CF809549
:1010B00080638D9308954E414E00496E66696E6956
:1010C00074790000302E300000404B4C0020A10706
:1010D000000050C3000088130000F401000000323B
:1010E0000000000500008000CCCCCC0C14AE470101
:1010F0009CC42000DC460300E353000063080000AA
:10110000D7000000150000001CC25367A5D4685327
:101110000024744915BE9A17CCBC8C2BBD3786357C
:10112000BBD00D920020E1F70895903071F00D9141
:101130001D912D913C9136952795179507959A9578
:10114000D1F73C932E931E930E930895D190E19086
:10115000F19001910895219131914191519108951A
:10116000FF0C90E89027110F9795F794092F089599
:10117000102FBD2CDE2CEF2CF02E11234AF4B0944E
:10118000D094E094F0949FEFB91AD90AE90AF90AC9
:101190000EE1FF2039F4FE2CED2CDB2CBB24085093
:1011A000C2F758C032F00A95BB0CDD1CEE1CFF1CC8
:1011B000F9CFEDDDD5CF502F2D2D3E2D4F2D612FA9
:1011C00008952DEC3CEC4CEC5DE366270FC0BEDFD0
:1011D000F2DFDD24EE2490E8F92E0FE307C0BBDF39
:1011E00005C02227332740E251E46627552351F1F9
:1011F000002381F1F7DD71F116270058505808944B
:10120000050B18F407FD03C025C007FD23C0469554
:1012100037952795F694E794D79422D0FF202AF0AB
:10122000DD0CEE1CFF1C015073F09D2D969548F0CF
:10123000DD203AF4EE202AF491E0D90E9927E91E38
:10124000F91E8ECF07C09FE7092FF92A9FEFD92EED
:10125000E92E0895DD24EE24FF24002711270895A8
:101260009F929924AA24BB2488E1D216E306F406AF
:1012700028F0D21AE30AF40A089401C08894991C51
:10128000AA1CBB1CDD0CEE1CFF1C8A9571F7D92C27
:10129000EA2CFB2C9F900895C89531960020089564
:1012A000FBDF202DF9DF302DF7DF402DF5DF502D4E
:1012B0000895041B150B260B370B089541E003C05E
:1012C00042E001C044E0E40F8827F81F829138E033
:1012D00098E1880F991F9D933A95D1F74A95B1F7F8
:1012E00000C088278D93089594E081918D939A95FD
:1012F000E1F7089509919191992351F08A95D9F7D1
:10130000319781918D930A9519F08823D1F708952B
:10131000E8CFE199FECFEEBBFFBB3196089591E097
:1013200001C092E07B3751F47FB7F894F2DF8D91E2
:101330008DBBE29AE19A9A95C9F77FBF7727089506
:1013400091E001C092E0E5DFE09A8DB38D939A952C
:10135000D1F70895689401C0E894AF93BF938D913D
:1013600016F0919102C098DF902D891718F011F4B2
:101370008823A9F7BF91AF910895000000400000B5
:10138000C8425B324A005B353B31480023330000E2
:10139000582D4163687365203A00206D6D005B4BEA
:1013A00000005B363B314800233400005B31343BA6
:1013B000314800003E005B32323B33364800616BFF
:1013C00074697600582D41636873653A00005B3894
:1013D0003B314800592D4163687365203A005B3901
:1013E0003B314800592D41636873653A00005B3119
:1013F000313B314800005A2D4163687365203A0043
:101400005B31323B314800005A2D41636873653AC5
:10141000000031002D002B005B313B3130480000D3
:101420004D65737373636869656265722041757396
:101430006C6573652053797374656D2056312E3158
:10144000612028323042697420326572204B6F6D02
:10145000706C656D656E742900005B323B313548F8
:101460000000A92048616E7320426F726E6772613E
:10147000656265722032303038005B31363B32486D
:101480000000C9CDCDCDCDCDCDCDCDCDCDCDCDCD2A
:10149000CDCDCDCDCDCDCDCDCDCDCDCDCDCDCDCD7C
:1014A000CDCDBB005B31373B32480000BA20622013
:1014B00020203D2062696E6165722020202020205E
:1014C000202020202020202020202020BA005B3156
:1014D000383B32480000BA20632020203D20636C56
:1014E0006561722020202020202020202020202024
:1014F000202020202020BA005B31393B32480000F8
:10150000BA20642020203D2064657A696D616C20DA
:1015100020202020202020202020202020202020CB
:10152000BA005B32303B32480000BA2065202020F0
:101530003D2065696E7269636874656E20202020A5
:1015400020202020202020202020BA005B32313BA8
:1015500032480000BA20662020203D206661737466
:1015600020726561642065696E2F6175732020208B
:1015700020202020BA005B32323B32480000BA20E3
:10158000722020203D2044757263686D6573736519
:10159000722F526164697573202020202020BA00C8
:1015A0005B32333B32480000BA20455343203D2094
:1015B00042696C6473636869726D206E6575206141
:1015C0007566626175656E20BA005B32343B3248E5
:1015D0000000C8CDCDCDCDCDCDCDCDCDCDCDCDCDDA
:1015E000CDCDCDCDCDCDCDCDCDCDCDCDCDCDCDCD2B
:1015F000CDCDBC00582D4163687365203A206E2E16
:10160000612E0000592D4163687365203A206E2ECB
:10161000612E00005A2D4163687365203A206E2EBA
:10162000612E00003E57656C6368652041636873F6
:101630006520617566204E756C6C2028782C792C9D
:101640007A2C61293F20000057656C636865204152
:10165000636873656E2073696E6420616E6765737D
:1016600063686C6F7373656E202878797A2C6C29A7
:021670003F0039
:00000001FF
